:1000000012C02CC02BC02AC029C028C027C026C0BF
:1000100025C024C023C022C021C020C01FC01EC0D4
:100020001DC01CC01BC011241FBECFE5D4E0DEBF25
:10003000CDBF11E0A0E6B0E0E0E6F9E002C0059037
:100040000D92A036B107D9F711E0A0E6B1E001C0EA
:100050001D92A436B107E1F7D7D380C4D1CFAD98B4
:10006000AC9A92B39F7092BB22B3982F907F922B41
:1000700092BBAC989AE19A95F1F7AC9A92B39F70C3
:1000800092BB92B38295807F982B92BBAC988AE604
:100090008A95F1F70895AD9AAC9A92B39F7092BB8E
:1000A00022B3982F907F922B92BBAC989AE19A95AD
:1000B000F1F7AC9A92B39F7092BB92B38295807F16
:1000C000982B92BBAC988AE68A95F1F708958FEF4A
:1000D00084BB80EF81BB929AAD98AC9A82B38F704B
:1000E00082BB82B3806382BBAC9820E137E2C90156
:1000F0000197F1F7AC9A82B38F7082BB82B38063B1
:1001000082BBAC98C9010197F1F7AC9A82B38F70AA
:1001100082BB82B3806382BBAC9820E43FE1C9011B
:100120000197F1F7AC9A82B38F7082BB959AAC9825
:10013000C9010197F1F7AC9A82B38F7082BB959A8F
:10014000AC98C9010197F1F7AC9A82B38F7082BB6A
:10015000979AAC98C9010197F1F7AC9A82B38F7066
:1001600082BBAC98C9010197F1F7AC9A82B38F704A
:1001700082BB82B3806C82BBAC98C9010197F1F756
:10018000AC9A82B38F7082BBAC98C9010197F1F72A
:10019000AC9A82B38F7082BB949AAC98C9010197D4
:1001A000F1F7AC9A82B38F7082BBAC98C90101970A
:1001B000F1F7AC9A82B38F7082BB82B3806382BB4B
:1001C000AC98C9010197F1F70895EF92FF920F9350
:1001D0001F93DF93CF93CDB7DEB760970FB6F89438
:1001E000DEBF0FBECDBFDE011196E0E5F1E080E19C
:1001F00001900D928150E1F780E831DF8E010F5FB1
:100200001F4F81E1E82EF12CEC0EFD1EF8018081DC
:1002100042DF0E5F1F4F0E151F05C1F780E593ECFF
:1002200028EC30E0F9013197F1F70197D9F76096A2
:100230000FB6F894DEBF0FBECDBFCF91DF911F91F7
:100240000F91FF90EF900895EF92FF920F931F93FD
:10025000DF93CF93CDB7DEB7A0970FB6F894DEBF8C
:100260000FBECDBFDE011196E0E4F1E080E1019028
:100270000D928150E1F7DE015196E0E3F1E080E17B
:1002800001900D928150E1F780E8E9DE8E010F5F69
:100290001F4F21E1E22EF12CEC0EFD1EF8018081B2
:1002A000FADE0E5F1F4F0E151F05C1F780ECD7DE7B
:1002B00091E2E92EF12CEC0EFD1EF8018081EBDEBF
:1002C0000E5F1F4F0E151F05C1F780E593EC28EC5C
:1002D00030E0F9013197F1F70197D9F7A0960FB601
:1002E000F894DEBF0FBECDBFCF91DF911F910F916C
:1002F000FF90EF900895EF92FF920F931F93DF937B
:10030000CF93CDB7DEB7A0970FB6F894DEBF0FBE80
:10031000CDBFDE011196E0E2F1E080E101900D92A7
:100320008150E1F7DE015196E0E1F1E080E10190DA
:100330000D928150E1F780E892DE8E010F5F1F4F32
:1003400041E1E42EF12CEC0EFD1EF8018081A3DECC
:100350000E5F1F4F0E151F05C1F780EC80DE31E2E6
:10036000E32EF12CEC0EFD1EF801808194DE0E5F71
:100370001F4F0E151F05C1F780E593EC28EC30E008
:10038000F9013197F1F70197D9F7A0960FB6F894D4
:10039000DEBF0FBECDBFCF91DF911F910F91FF90B8
:1003A000EF900895EF92FF920F931F93DF93CF93F7
:1003B000CDB7DEB7A0970FB6F894DEBF0FBECDBFA6
:1003C000DE011196E0E0F1E080E101900D928150B4
:1003D000E1F7DE015196E0EFF0E080E101900D924F
:1003E0008150E1F780E83BDE8E010F5F1F4F61E136
:1003F000E62EF12CEC0EFD1EF80180814CDE0E5F26
:100400001F4F0E151F05C1F780EC29DE51E2E52EC6
:10041000F12CEC0EFD1EF80180813DDE0E5F1F4FBA
:100420000E151F05C1F780E593EC28EC30E0F901CB
:100430003197F1F70197D9F7A0960FB6F894DEBF80
:100440000FBECDBFCF91DF911F910F91FF90EF9025
:100450000895EF92FF920F931F93DF93CF93CDB741
:10046000DEB7A0970FB6F894DEBF0FBECDBFDE019A
:100470001196E0EEF0E080E101900D928150E1F7FD
:10048000DE015196E0EDF0E080E101900D928150A7
:10049000E1F780E8E4DD8E010F5F1F4FE1E1EE2E12
:1004A000F12CEC0EFD1EF8018081F5DD0E5F1F4F73
:1004B0000E151F05C1F780ECD2DD71E2E72EF12C9D
:1004C000EC0EFD1EF8018081E6DD0E5F1F4F0E155C
:1004D0001F05C1F780E593EC28EC30E0F901319776
:1004E000F1F70197D9F7A0960FB6F894DEBF0FBECB
:1004F000CDBFCF91DF911F910F91FF90EF900895A5
:10050000EF92FF920F931F93DF93CF93CDB7DEB798
:1005100060970FB6F894DEBF0FBECDBFDE01119617
:10052000E0ECF0E080E101900D928150E1F780E88D
:1005300096DD8E010F5F1F4FF1E1EF2EF12CEC0ED7
:10054000FD1EF8018081A7DD0E5F1F4F0E151F05F0
:10055000C1F780E593EC28EC30E0F9013197F1F731
:100560000197D9F760960FB6F894DEBF0FBECDBFE6
:10057000CF91DF911F910F91FF90EF900895EF922F
:10058000FF920F931F93DF93CF93CDB7DEB76097A2
:100590000FB6F894DEBF0FBECDBFDE011196E0EBC3
:1005A000F0E080E101900D928150E1F780E857DDA5
:1005B0008E010F5F1F4FA1E1EA2EF12CEC0EFD1E04
:1005C000F801808168DD0E5F1F4F0E151F05C1F712
:1005D00080E593EC28EC30E0F9013197F1F70197D1
:1005E000D9F760960FB6F894DEBF0FBECDBFCF919E
:1005F000DF911F910F91FF90EF900895EF92FF927E
:100600000F931F93DF93CF93CDB7DEB760970FB6ED
:10061000F894DEBF0FBECDBFDE011196E8EAF0E030
:1006200088E001900D928150E1F7DE011996E0EA31
:10063000F0E088E001900D928150E1F780E80FDD55
:100640008E010F5F1F4F89E0E82EF12CEC0EFD1E8E
:10065000F80181918F011FDD0E151F05C9F780EC90
:10066000FEDCB1E1EB2EF12CEC0EFD1EF8018191C8
:100670008F0111DD0E151F05C9F780E593EC28ECFD
:1006800030E0F9013197F1F70197D9F760960FB68D
:10069000F894DEBF0FBECDBFCF91DF911F910F91B8
:1006A000FF90EF900895EF92FF920F931F93DF93C7
:1006B000CF93CDB7DEB760970FB6F894DEBF0FBE0D
:1006C000CDBF80E8CCDCDE011196E0E9F0E080E10E
:1006D00001900D928150E1F78E010F5F1F4F91E164
:1006E000E92EF12CEC0EFD1EF8018081D4DC0E5FAA
:1006F0001F4F0E151F05C1F780E593EC28EC30E085
:10070000F9013197F1F70197D9F760960FB6F89490
:10071000DEBF0FBECDBFCF91DF911F910F91FF9034
:10072000EF9008958CB59DB59C0140E050E020937A
:10073000600130936101409362015093630121375E
:100740006CE1360760E0460760E0560710F43DDDD7
:100750000895DA01C90181579C41A040B0408157FA
:100760009C41A040B04010F46FDD0895DA01C9014A
:10077000825E9843A040B04081579C41A040B04069
:1007800010F4B9DD0895DA01C90183559545A040FB
:10079000B04081579C41A040B04010F403DE089562
:1007A000DA01C901845C9147A040B04081579C4167
:1007B000A040B04010F44DDE0895DA01C901855320
:1007C0009E48A040B04081579C41A040B04010F4EA
:1007D00097DE0895DA01C901865A9A4AA040B040CE
:1007E00081579C41A040B04010F4C9DE08952751C4
:1007F000374C4040504021573C414040504010F45D
:10080000FDDE089550DF08956F927F928F929F9240
:10081000AF92BF92CF92DF92EF92FF920F931F930E
:10082000DF93CF93CDB7DEB7E0970FB6F894DEBF76
:100830000FBECDBF1FBC81E08EBD1DBC1CBCDE0148
:100840005196E0E8F0E080E101900D928150E1F7EF
:10085000DE019196E0E7F0E080E101900D92815099
:10086000E1F7DE011196E8E6F0E088E001900D92F4
:100870008150E1F7DE011996E0E6F0E088E00190B2
:100880000D928150E1F723DC80E8E9DB8E010F5EF9
:100890001F4F71E2E72EF12CEC0EFD1EF801808156
:1008A000FADB0E5F1F4F0E151F05C1F780ECD7DB7B
:1008B00061E3E62EF12CEC0EFD1EF8018081EBDBEE
:1008C0000E5F1F4F0E151F05C1F780E29EE428EC56
:1008D00030E0F9013197F1F70197D9F781E0BFDBFB
:1008E00080E197E20197F1F73E010894611C711CC9
:1008F00059E0E52EF12CEC0EFD1E41E1842E912CE9
:100900008C0E9D1E30E1A32E37E2B32E28ECC22EB2
:10091000D12C14C080E8A3DB8301F80181918F0101
:10092000BADB0E151F05C9F780EC99DB8701F801CA
:1009300081918F01B0DB08151905C9F78299EACFBB
:1009400081E08DDBC5010197F1F7ECDE80E593ECEA
:10095000F6013197F1F70197D9F7F0CFF894FFCF6F
:10096000A86FBF70C763B82143BE706F63B820B86B
:10097000540052005500C100BA006100210020005F
:10098000A8007000B800B3006500BF002C00C700CD
:100990002000200048006500BF002100200020004A
:1009A000B3206FBFBE7963BA4DBD6520BE6F706165
:1009B000A5002000B7006100C0006500BC00210058
:1009C000E00061002000B20070006F006300C4000E
:1009D000E0006500BB006100B9002E002E002E0073
:1009E0002000480079002E002E002E002E0020004E
:1009F0002000BD006100E3006F003F0021002000E7
:100A000054006500B200650020006F00BD006F005B
:100A1000E30065007000B6006100BF00C400210063
:100A20002000200054006100BA00200020002000B7
:100A300020006300BF006F00B800BF00210020004D
:100A40002000200020004800650020002000200039
:100A5000200020002000E000610021002000200094
:00000001FF
